:020000040800F2
:100000009008002045010008950A00088D0A0008A4
:10001000910A00088D010008B31D000800000000CF
:10002000000000000000000000000000E1150008D2
:10003000710900080000000041100008491700087D
:100040005F0100085F0100085F0100085F01000810
:100050005F0100085F0100085F0100085F01000800
:100060005F0100085F0100085F0100085F010008F0
:100070005F0100085F0100085F0100085F010008E0
:100080005F0100085F0100085F0100085F010008D0
:100090005F0100085F0100085F0100085F010008C0
:1000A0005F0100085F0100085F0100085F010008B0
:1000B0005F010008AD1700085F0100085F0100083C
:1000C0005F0100085F0100085F0100085F01000890
:1000D0005F0100081919000865190008491A00088D
:1000E0005F0100085F0100085F0100085F01000870
:1000F0005F0100085F0100085F0100085F01000860
:100100005F0100085F0100085F0100085F0100084F
:100110005F0100085F0100085F0100085F0100083F
:100120005F0100085F0100085F0100085F0100082F
:10013000DFF80CD000F018F800480047B11E0008A6
:10014000900800200648804706480047FEE7FEE783
:10015000FEE7FEE7FEE7FEE7FEE7FEE7FEE7FEE777
:100160004D17000831010008064C074D06E0E06815
:1001700040F0010394E8070098471034AC42F6D3EE
:10018000FFF7DAFF5C1F00087C1F000800BFFEE7D6
:1001900010B502460B460020002104E0545C0444E4
:1001A000E0B24C1CE1B29942F8DBC443E0B2441C1B
:1001B000E0B210BD10B5344800780A281DD133488C
:1001C000007833490978884217D13048407830495F
:1001D0004978884211D12D48007A2D49097A884200
:1001E0000BD12A48407A2A49497A884205D12948C0
:1001F000008840F40040274908802648008810F411
:10020000004F3FD0002024490870204800794870F2
:100210001E48407988701D488079C8701B48C07995
:100220000871084600781D4908701B4840784870DE
:100230001948807888701848C078C87016480079C6
:100240000871174800686FEA00001649C1F880017C
:100250004FF40071144800F017FC4FF4FA7001F0ED
:10026000D3FD4FF40071104800F00CFC0D48D0F89D
:100270008001C0430A4908604FF00000024908703D
:100280000449088010BD00000700002090010020F4
:100290000E0000200800002018000020430000206D
:1002A00080012242000022420010014010B588B0B7
:1002B00056480078002831D0002054490870FC20AE
:1002C000534908701120487052480078887051488E
:1002D0004078C8704F48807808714E48C07848719F
:1002E0004C480079887107214948FFF751FF484978
:1002F000C8710020484908604FF0FF024FF0E1014B
:1003000000F0EAFD0823424AA821002000F0A6FDE3
:10031000002000F06BFC0120404908703F48007845
:10032000002871D03E480088B0F5FA6F6CDC3D487B
:100330000068002868D1694600F022FD0446204686
:1003400001F050F904F0400040285DD100208DF804
:100350000700354800686FEA00003449C1F88001A1
:100360004FF00701684601F047F99DF8010029495F
:100370000978884234D19DF802002649497888429C
:100380002ED19DF8030023498978884228D19DF811
:1003900004002049C978884222D19DF805001D49F2
:1003A000097988421CD11D48007801280ED11B48CC
:1003B0000078401C1949087012201549487008231C
:1003C0000A46A821002000F049FD1DE00020134945
:1003D0000870134908800E21154801F00DF913E04B
:1003E00000200D4908604FF01100094948704FF096
:1003F00008030A464FF0A8014FF0000000F02EFD60
:1004000001200C49C1F8980108B010BD4800002037
:100410001E00002043000020988121423E00002061
:1004200040000020000121428001224200002242BF
:10043000C40300200080214210B5D14800780E2866
:100440001BD1D048407BFB2817D1CE480078FA2832
:100450000DD1CB480078401ECA49085CFB2806D164
:10046000C948008840F40040C74908802DE00020BA
:10047000C3490870C449088027E0C248007B103097
:10048000BF490978884217D1BE480078FA280DD1B3
:10049000BB480078401EBB49085CFB2806D1BA481F
:1004A000008840F40040B84908800EE00020B449BC
:1004B0000870B549088008E0B1480078182804DDC4
:1004C0000020AF490870B0490880AF48008810F498
:1004D000004F71D0AB488079AC498871A948C17987
:1004E000AA48C171A748017AA8480172A548417A73
:1004F000A6484172A348807AA44988720846807948
:10050000A3498871A148C179A148C1719F48017A66
:100510009F4801729D48417A9D4841729B48807A6C
:1005200078285FD012DC71283FD008DC212820D049
:10053000222825D025282AD026287DD12EE07328F0
:100540003BD0742840D07528F7D144E0A22874D05D
:1005500008DC82284DD0942852D0A02857D0A1285A
:10056000EBD199E0A32869D0A42868D0A528E4D1CC
:10057000F4E088A001F020FC002084498872F5E0B6
:1005800086A001F019FC002080498872EEE087A067
:1005900001F012FC00207D498872E7E087A001F09D
:1005A0000BFC002079498872E0E088A001F004FC8F
:1005B000002076498872D9E0E0E087A001F0FCFBDA
:1005C000002072498872D1E086A001F0F5FB00207E
:1005D0006E498872CAE086A001F0EEFB00206B49EC
:1005E0008872C3E085A001F0E7FB002067498872AC
:1005F000BCE085A001F0E0FB002064498872B5E012
:1006000083A001F0D9FB002060498872AEE05F480A
:100610008079834988715D48C1798148C1715B489F
:10062000017A7F4801725948417A7D4841725748A2
:10063000807A7B49887203E097E031E080E086E0D1
:100640005048407B514948734E48817B4F488173E5
:100650004C48C17B4D48C1734A48017C4B480174EA
:100660004848417C49484174407B6E49087047487E
:10067000807B48704548C07B88704448007CC870C7
:100680004248407C08710120674908700020674992
:1006900008803E49887269E000203C49887265E024
:1006A0003A488079624988713848C1796048C17197
:1006B0003648017A5E4801723448417A5C4841729A
:1006C0003248807A5A4988720120C872062008731D
:1006D0000020487357480178554881735548417840
:1006E0005348C17353488178514801745148C178C7
:1006F0004F4841744F4801794D48817402204C495C
:10070000C874062008750020487546480178484896
:100710008175444841784648C175424881784448CB
:1007200001764048C178424841763E4801794048C8
:1007300081761E2100F060FF00201449887215E0C8
:100740003DA001F039FB0020104988720EE03FA067
:1007500001F032FB00200D49887207E03EA001F055
:100760002BFB00200949887200E000BF00BF002079
:1007700005490880024908703C49087010BD000016
:1007800003000020C800002004000020FC0200201C
:100790009802002052657365740A0000476574462C
:1007A00069726D76657273696F6E0A005365745273
:1007B000656164657249440A00000000476574522F
:1007C000656164657249440A0000000044656C5725
:1007D000686974650A0000004F70656E5768697437
:1007E000650A0000436C6F736557686974650A0099
:1007F00041646457686974650A000000476574576E
:10080000686974650A00000048656172740A000036
:10081000476574576869746553746174650A0000AC
:10082000C4030020430000204800002040000020B6
:1008300060030020180000205570646174654669EB
:10084000726D76657273696F6E0A0000557064612F
:1008500074654669726D0A00557064617465466915
:10086000726D53746174650A00000000020000207C
:10087000FA203B4908701020487000208870002141
:100880003748C170017141710020354988710021DC
:100890003348C1710172417200203149C87400218E
:1008A0002F480175FB202E494875FA202D49087004
:1008B000102048700020887000212A48C170017102
:1008C000417100202749887100212648C1710172B9
:1008D00041720020234981F84B000021214880F813
:1008E0004C10FB201F4981F84D00FA201E4908706A
:1008F000102048700020887000211B48C1700171D1
:10090000417100201849887100211748C171017296
:10091000417200201449C876002113480177FB205A
:1009200011494877FA2011490870102048700020BA
:10093000887000210D48C1700171417100200B4980
:10094000887100210948C171017241720020074974
:10095000C872002105480173FB20044948737047A1
:1009600098020020FC02002060030020C403002045
:1009700070472DE9F04102460025002600200023A3
:100980000024002791F803C00CF00F0591F803C074
:100990001CF0100F03D091F802C04CEA050591F845
:1009A00000C0BCF1000F31D0146800202BE04FF0E4
:1009B000010C0CFA00F3B1F800C00CEA03069E42E9
:1009C00020D183004FF00F0C0CFA03F7BC4305FA5B
:1009D00003FC4CEA040491F803C0BCF1280F06D1D3
:1009E0004FF0010C0CFA00FCC2F814C00AE091F8B8
:1009F00003C0BCF1480F05D14FF0010C0CFA00FC0C
:100A0000C2F810C0401C0828D1D31460B1F800C04F
:100A1000BCF1FF0F34DD546800202EE000F1080C1B
:100A20004FF0010808FA0CF3B1F800C00CEA030615
:100A30009E4221D183004FF00F0C0CFA03F7BC4308
:100A400005FA03FC4CEA040491F803C0BCF1280F3A
:100A500005D100F1080C08FA0CF8C2F8148091F8DE
:100A600003C0BCF1480F07D100F1080C4FF001089A
:100A700008FA0CF8C2F81080401C0828CED3546045
:100A8000BDE8F081416170470161704700BFFEE73A
:100A900000BFFEE7704700007CB5054612A103C900
:100AA000CDE900010821284600F072FD05236A46C1
:100AB0003021284600F0D2F905236A461021284645
:100AC00000F0F0F8002406E01DF80400A52800D08E
:100AD00003E0601CC4B2052CF6DB00BF052C01D07E
:100AE00001207CBD0020FCE7A5A5A5A5A500000070
:100AF00008B501211C2000F0B5FA4020ADF8000037
:100B000010208DF8030003208DF80200694631485B
:100B1000FFF72FFF40212F48FFF7B6FF1020ADF859
:100B2000000069462C48FFF724FF10212A48FFF7F0
:100B3000ABFF0120ADF8000048208DF80300032032
:100B40008DF8020069462448FFF713FF4FF4007048
:100B5000ADF8000010208DF8030003208DF802008E
:100B600069461C48FFF705FF4FF400711948FFF76D
:100B70008BFF4FF48050ADF8000069461548FFF731
:100B8000F8FE4FF480511348FFF77EFF4FF480705A
:100B9000ADF8000048208DF8030003208DF8020016
:100BA00069460C48FFF7E5FE00F020FC00F0DCFB96
:100BB00000200A4908604FF001000949C1F890017E
:100BC0004FF00000074908604FF001000649C1F8E6
:100BD000B00108BD000C014000080140988121428D
:100BE00000002142A48121420080214210B5044628
:100BF0001CB900202749086002E00020264908604F
:100C00004FF001024FF02301204600F065F9032365
:100C1000224A2A21204600F021F90323204A3021CC
:100C2000204600F01BF901222121204600F054F952
:100C300001222221204600F04FF92A2225212046B8
:100C400000F04AF907222621204600F045F90F223C
:100C50002021204600F040F906223D21204600F0E8
:100C60003BF901223C21204600F036F97022272171
:100C7000204600F031F9FF22E221204600F02CF955
:100C80001CB901200349086002E001200249086004
:100C900010BD000098812142A4812142551F000807
:100CA000501F00082DE9F0478046894615461E462C
:100CB000B8F1000F16D10020174908604946404698
:100CC00000F012FC0746002406E0FF21404600F039
:100CD0000BFC2855601CC4B2B442F6DB01200E495F
:100CE000086015E000200D4908604946404600F0C4
:100CF000FBFB0746002406E0FF21404600F0F4FB22
:100D00002855601CC4B2B442F6DB012003490860D8
:100D10003846BDE8F087000090012142B0812142B1
:100D200070B505460E4685B9002011490860314668
:100D3000284600F0D9FBFF21284600F0D5FB0446E9
:100D400001200C49C1F890010FE000200A49086019
:100D50003146284600F0C8FBFF21284600F0C4FBBE
:100D6000044601200549C1F8B001204670BD0000CD
:100D70009001214200002142B081214200802142A5
:100D800070B506460D461021304600F001FC0721E3
:100D90003046FFF7C5FF044622462721304600F0C3
:100DA0009BF814F0400F0AD007232A4661213046F1
:100DB000FFF778FFFF22E221304600F08DF8204651
:100DC00070BD000010B504461CB900201F49086022
:100DD00002E000201E4908604FF001024FF023019D
:100DE000204600F079F803231A4A3021204600F00B
:100DF00035F80323184A2A21204600F02FF8012253
:100E00002121204600F068F801222221204600F02E
:100E100063F81A222421204600F05EF82A222521B8
:100E2000204600F059F807222621204600F054F809
:100E30000E222021204600F04FF81CB90120034962
:100E4000086002E001200249086010BD988121423B
:100E5000A4812142501F0008551F00082DE9F047CA
:100E60008046894615461E46B8F1000F16D100206F
:100E7000174908604946404600F036FB0746002403
:100E800006E015F8011B404600F02EFB601CC4B2C2
:100E9000B442F6DB01200E49086015E000200D4940
:100EA00008604946404600F01FFB0746002406E064
:100EB00015F8011B404600F017FB601CC4B2B44299
:100EC000F6DB0120034908603846BDE8F0870000E2
:100ED00090012142B08121422DE9F04104460E46A5
:100EE000154684B90020114908603146204600F0BB
:100EF000FBFA07462946204600F0F6FA01200C4985
:100F0000C1F890010FE000200A49086031462046F0
:100F100000F0EAFA07462946204600F0E5FA0120EB
:100F20000549C1F8B0013846BDE8F0819001214281
:100F300000002142B08121420080214208B54FF4D7
:100F4000C06000F073F826208DF8000001208DF8B5
:100F5000010002208DF8020001208DF80300684690
:100F600000F02AF827208DF8000001208DF80100FC
:100F70008DF802008DF80300684600F01DF825206A
:100F80008DF8000000208DF8010001208DF802008E
:100F90008DF80300684600F00FF81D208DF8000062
:100FA00000208DF801008DF8020001208DF803006B
:100FB000684600F001F808BD70B5002100230F223B
:100FC000C4780CB3164C246804F4E064C4F5E064FF
:100FD000210AC1F10403CA40447804FA03F1847879
:100FE0001440214309010F4C0678A155047804F000
:100FF0001F050124AC4005786D114FF0E02606EB8B
:101000008505C5F8004109E0047804F01F050124B6
:10101000AC40054D0678761145F8264070BD0000BD
:101020000CED00E000E400E080E100E00249014353
:10103000024A1160704700000000FA050CED00E064
:101040007047000029B1064AD2690243044BDA61B5
:1010500004E0034AD2698243014BDA617047000021
:101060000010024029B1064A92690243044B9A617A
:1010700004E0034A92698243014B9A617047000081
:101080000010024010B500F033F84FF4803000F04B
:10109000F1F800F04DF90446012C1ED1002000F0BB
:1010A000DDF8002000F018F9A00200F009F94FF473
:1010B000E011200400F022F9012000F019F900BF2E
:1010C000392000F0A5F80028FAD0022000F024F919
:1010D00000BF00F0BBF80828FBD1012144F20D004D
:1010E000FFF7C0FF01210220FFF7ACFF10BD000099
:1010F0000F48006840F001000D490860084640684C
:101100000C4908400A494860084600680A490840F6
:10111000074908600846006820F4802008600846F7
:10112000406820F4FE0048604FF41F00886070475C
:10113000001002400000FFF8FFFFF6FE30B500216E
:101140000022002400232D4D6D6805F00C0121B113
:10115000042905D0082923D105E0294D056022E0A6
:10116000274D05601FE0254D6D6805F47012234D75
:101170006D6805F48034022505EB92421CB9214DBF
:10118000554305600BE01D4D6D6815F4003F03D01D
:101190001C4D5543056002E0194D5543056002E0C2
:1011A000174D056000BF00BF144D6D6805F0F001DC
:1011B0000909154D6B5C0568DD4045600F4D6D6894
:1011C00005F4E061090A104D6B5C4568DD408560FF
:1011D0000A4D6D6805F46051C90A0B4D6B5C45689A
:1011E000DD40C560054D6D6805F44041890B074D34
:1011F0006B5CC568B5FBF3F5056130BD00100240BE
:1012000000127A0000093D0049000020590000202A
:1012100010B501460022002300204A11012A02D104
:10122000094C236806E0022A02D1074C236A01E038
:10123000054C636A01F01F02012494401C4201D056
:10124000012000E0002010BD00100240024840686C
:1012500000F00C0070470000001002400146002022
:10126000034A506820F0F0000843506070470000C7
:10127000001002401149096821F480310F4A1160C1
:101280001146096821F480211160B0F5803F03D038
:10129000B0F5802F0ED106E00849096841F480318D
:1012A000064A116007E00549096841F4A021034A94
:1012B000116000E000BF00BF704700000010024056
:1012C00001460020034A506820F4E0600843506063
:1012D000704700000010024001460020034A506899
:1012E00020F4605040EAC100506070470010024096
:1012F0000149086670470000000042420246002093
:10130000044B586820F47C1042EA01031843014B57
:10131000586070470010024001460020034A5068A0
:1013200020F00300084350607047000000100240A6
:1013300038B5002000900024002500BF3120FFF7C1
:1013400067FF05460098401C00900098B0F5A06F1C
:1013500001D0002DF2D03120FFF75AFF08B101244F
:1013600000E00024204638BD00B587B0012141F2DD
:101370000500FFF777FEE020ADF8180018208DF883
:101380001B0003208DF81A0006A91648FFF7F1FA92
:10139000E0211448FFF778FB0020ADF804004FF47B
:1013A0008270ADF806000020ADF80800ADF80A0024
:1013B000ADF80C004FF40070ADF80E001820ADF839
:1013C00010000020ADF812000720ADF8140001A9AC
:1013D000054800F06BF80121034800F04DF807B014
:1013E00000BD0000000801400030014000B587B09A
:1013F00001218803FFF726FE01210920FFF732FEB5
:101400004FF46040ADF8180018208DF81B00032041
:101410008DF81A0006A91648FFF7ABFA4FF46041A1
:101420001348FFF731FB0020ADF804004FF4827041
:10143000ADF806000020ADF80800ADF80A00ADF8E0
:101440000C004FF40070ADF80E001820ADF810003D
:101450000020ADF812000720ADF8140001A90548DE
:1014600000F024F80121034800F006F807B000BDA1
:10147000000C01400038004021B1028842F04002D7
:10148000028004E002884FF6BF731A400280704762
:101490000246002013890B4201D0012000E0002009
:1014A00070470146888970478181704710B50022D6
:1014B000028802F441520B884C8823438C882343D2
:1014C000CC8823430C8923434C8923438C892343B1
:1014D000CC8923431A430280838B4FF2FF7423404D
:1014E00083830B8A038210BD2DE9F04106460F4627
:1014F00026BB06E0601CC4B2C82C02DB0020BDE89D
:10150000F08102212048FFF7C3FF0028F2D03946BE
:101510001D48FFF7C9FF002405E0601CC4B2C82CB9
:1015200001DB0020EBE701211748FFF7B1FF00289E
:10153000F3D01548FFF7B5FFC5B222E005E0601C07
:10154000C4B2C82C01DB0020D9E702210F48FFF705
:101550009FFF0028F3D039460C48FFF7A5FF002471
:1015600005E0601CC4B2C82C01DB0020C7E70121E4
:101570000648FFF78DFF0028F3D00448FFF791FFDE
:10158000C5B22846BBE700000030014000380040EB
:1015900070B505460C467DB90F4800884FF6C771F7
:1015A00008400D4908800846008820430880012132
:1015B0000A48FFF761FF0EE0084800884FF6C77140
:1015C0000840064908800846008820430880012119
:1015D0000248FFF751FF70BD003001400038004065
:1015E0007047000010B504460249204600F010F88C
:1015F00010BD00000038014070B504460D46034A96
:101600002946204600F014F870BD00000038014063
:1016100070B504460D4600BF8021284600F0F8FA58
:101620000028F9D02146284600F0BFFB012070BDFC
:101630002DE9F04104460D46164614B90120BDE8D7
:10164000F0810AE014F8017B31463846FFF7E0FFED
:1016500008B90020F3E7681E85B2002DF2D1012001
:10166000EDE710B500F002F810BD00000CB5002049
:10167000019000903248006840F4803030490860A2
:1016800000BF2F48006800F4003000900198401C13
:101690000190009818B90198B0F5A06FF1D12848D1
:1016A000006810F4003F02D00120009001E000200B
:1016B00000900098012842D12248006840F01000B4
:1016C000204908600846006820F0030008600846CA
:1016D000006840F0020008601948406818494860F6
:1016E0000846406848600846406840F480604860AA
:1016F0000846406820F47C1048600846406840F482
:10170000E81048600846006840F08070086000BF3C
:101710000B48006810F0007FFAD00948406820F0BC
:101720000300074948600846406840F002004860EE
:1017300000BF0348406800F00C000828F9D10CBD38
:1017400000100240002002407047000010B513480E
:10175000006840F0010011490860084640681049DF
:1017600008400E494860084600680E4908400B4989
:1017700008600846006820F4802008600846406839
:1017800020F4FE0048604FF41F008860FFF769FFF7
:101790004FF000600449086010BD000000100240D6
:1017A0000000FFF8FFFFF6FE08ED00E010B5012194
:1017B000084800F044F858B10121064800F030F81C
:1017C00005480088401C044908800120034908702E
:1017D00010BD000000040040400000204200002036
:1017E0003EB505460C4601210220FFF72BFCADF863
:1017F0000450ADF800400020ADF80600ADF802003E
:101800006946064800F036F801221146034800F008
:1018100027F80121014800F006F83EBD0004004011
:10182000CA430282704721B1028842F0010202805D
:1018300004E002884FF6FE731A400280704730B50C
:101840000246002000230024158A05EA0103958939
:1018500005EA010413B10CB1012000E0002030BD05
:101860001AB183890B43838102E083898B4383818F
:1018700070470000002202881D4B98420ED01D4B7D
:1018800098420BD0B0F1804F08D01B4B984205D046
:101890001A4B984202D01A4B984204D14FF68F73DC
:1018A0001A404B881A43174B984207D0164B984260
:1018B00004D04FF6FF431A40CB881A4302808B882E
:1018C00083850B8803850A4B98420BD0094B9842BD
:1018D00008D00E4B984205D00D4B984202D00D4BCC
:1018E000984201D10B7A038601238382704700005E
:1018F000002C01400034014000040040000800407A
:10190000000C004000100040001400400040014066
:10191000004401400048014010B540F225510D48F7
:1019200000F083F9A8B140F225510A4800F0C7F849
:10193000084800F035FAC4B22146074800F035FAED
:10194000064807490978445405480078401C044972
:10195000087010BD0038014000440040C80000205D
:101960000300002010B540F22551124800F05DF947
:1019700088B140F225510F4800F0A1F80D4800F061
:101980000FFAC4B20C480D49097844540B4800784A
:10199000401C0A4908700821064800F039F901285E
:1019A00006D10821034800F081F8024800F0F8F958
:1019B00010BD000000440040580200200B00002031
:1019C00010B586B0044601210520FFF74BFB01212D
:1019D0004804FFF737FB0420ADF8140003208DF80E
:1019E000160018208DF8170005A91548FEF7C1FF4D
:1019F0000820ADF8140004208DF8170005A9104840
:101A0000FEF7B7FF01940020ADF80800ADF80A001A
:101A1000ADF80C00ADF810000C20ADF80E0001A9D7
:101A2000084800F051F9012240F22551054800F024
:101A300026F90121034800F051F806B010BD00005E
:101A4000000801400044004010B540F22551144800
:101A500000F0EBF8B0B140F22551114800F02FF83A
:101A60000F4800F09DF9C4B20E480F49097844545C
:101A70000D480078401C0C4908700846007800F0BA
:101A80000F0008700821064800F0C2F8012806D1AE
:101A90000821034800F00AF8014800F081F910BD60
:101AA00000480040900100200700002001F400726F
:101AB000B2F5007F00D100BFCA430280704710B565
:101AC00000220023A1F510646A3C00D100BF0A1275
:101AD00001249440A3B2DC43048010BD21B182896B
:101AE00042F40052828104E082894DF6FF731A406D
:101AF0008281704700B585B0012144F20400FFF7F0
:101B0000B1FA4FF40070ADF8000003208DF8020028
:101B100018208DF8030069463948FEF72AFF4FF474
:101B20008060ADF8000004208DF803006946344859
:101B3000FEF71FFF4FF4E13001900020ADF80800E0
:101B4000ADF80A00ADF80C00ADF810000C20ADF8AF
:101B50000E0001A92B4800F0B7F8012240F22551F0
:101B6000284800F08CF801212648FFF7B7FF012133
:101B70008804FFF767FA01210820FFF773FA4FF492
:101B80008060ADF8000003208DF8020018208DF869
:101B9000030069461C48FEF7ECFE4FF40060ADF808
:101BA000000004208DF8030069461748FEF7E1FEA7
:101BB0004FF4965001900020ADF80800ADF80A00EF
:101BC000ADF80C00ADF810000C20ADF80E0001A926
:101BD0000E4800F079F801A90C4800F075F80122D0
:101BE00040F22551094800F04AF801210748FFF763
:101BF00075FF40210348FFF759FF05B000BD000005
:101C00000008014000380140000C0140004800403D
:101C100002460020B1F5007F00D100BF13880B42BF
:101C200001D0012000E00020704770B5024600247A
:101C3000002300250020A1F510666A3E00D100BFF8
:101C4000C1F3421501F01F03012606FA03F3012D2B
:101C500002D19689334006E0022D02D1168A334024
:101C600001E0968A33400C12012606FA04F4168825
:101C7000344013B10CB1012000E0002070BDF0B57C
:101C800003460024002600250020A1F510676A3FC6
:101C900000D100BF1846C1F3421401F01F0601270E
:101CA00007FA06F5012C01D10C3004E0022C01D119
:101CB000103000E014301AB107682F43076002E0CB
:101CC0000768AF430760F0BD2DE9F04786B00546D1
:101CD0000E460024A24600BFA1460027B08900B1ED
:101CE00000BF2F462C8A4CF6FF700440F088044356
:101CF0002C82AC894EF6F3100440B0883189084339
:101D0000718908430443AC81AC8A4FF6FF4004401C
:101D1000B0890443AC8201A8FFF710FA1F4887423C
:101D200002D1DDF810A001E0DDF80CA0A88910F4C4
:101D3000004F08D00AEBCA0000EB0A1031684900D6
:101D4000B0FBF1F807E00AEBCA0000EB0A103168BB
:101D50008900B0FBF1F86420B8FBF0F00401200921
:101D6000642101FB1089A88910F4004F08D03220AB
:101D700000EBC900B0FBF1F000F00700044308E0FD
:101D8000322000EB09106421B0FBF1F000F00F00ED
:101D900004432C8106B0BDE8F08700000038014004
:101DA00001468888C0F308007047C1F308028280AA
:101DB000704700BFFEE70000014A024900F013B877
:101DC000351E00086000002002E008C8121F08C18C
:101DD000002AFAD170477047002001E001C1121FAC
:101DE000002AFBD170472DE9F04116460F46044604
:101DF000002503E03946B0476D1C641C207800289C
:101E0000F8D12846BDE8F08110B502460BE0C820A5
:101E100007E0122101E04B1E99B20029FBDC431EB2
:101E200098B20028F5DC1300A2F10104A2B2EED1B1
:101E300010BD000070B504460D46E0B205490880AB
:101E400000BF40210348001FFFF7E2FE0028F8D042
:101E5000204670BD0438014008B501211020FFF76D
:101E600001F90120ADF8000010208DF803000320D7
:101E70008DF8020069460D48FEF77BFD01210B48F5
:101E8000FEF702FE4FF40070ADF8000010208DF850
:101E9000030003208DF8020069460448FEF769FD3F
:101EA0004FF400710148FEF7EDFD08BD0010014040
:101EB000FFF7E8F8FFF742F841F61F410920FFF766
:101EC0008FFCFFF7C9FFFFF715FE4FF4E130FFF776
:101ED00077FDFEF70DFE02E017A0FFF76DFF002073
:101EE000FEF7DAFD0028F7D102E013A0FFF764FF48
:101EF0000120FEF7D1FD0028F7D1FEF7B9FC12480A
:101F000000686FEA00001149C1F880014FF4FA70CF
:101F1000FFF77AFF0D48D0F88001C0430B49C1F8A4
:101F200080010120FEF74EFF05E0FEF743F9FEF7C2
:101F3000BDF9FEF781FAF8E754686520322E344780
:101F4000204572726F7221008001224200002242FD
:101F50003443101001344310100100007C1F0008AE
:101F60000000002064000000C81D0008E01F0008F9
:101F7000640000202C080000D81D000800000000AC
:101F800000000000000000000000D1D1E0D00000FF
:101F90000000D2D200000000000031323334353668
:101FA00037383931323334353637383900000000AC
:101FB0000000000000000000000000000000000021
:101FC0000000000000000000000102030401020301
:101FD00004060708090204060800000000000000CB
:0400000508000131BD
:00000001FF
